
 TIMER

 Start     Length     Name                   Class
 0001:0000 00168H     INIT_CODE              CODE
 0002:0000 000B4H     FIXED_TEXT             CODE
 0003:0000 005DFH     FIXED_286              CODE
 0004:0000 0021CH     _DATA                  DATA

 Origin   Group
 0004:0   DGROUP

 Address   Export                  Alias

 0002:0038 DriverProc              DriverProc
 0001:0000 WEP                     WEP

  Address         Publics by Name

 0000:0000  Imp  AllocCStoDSAlias     (KERNEL.170)
 0004:01D2       CurTime
 0001:0000       Disable
 0001:0145       Disable286
 0000:0000  Imp  DriverCallback       (MMSYSTEM.31)
 0002:0038       DriverProc
 0004:01E4       dTickUpdate
 0001:002A       Enable
 0001:013B       Enable286
 0004:0014       Events
 0000:0000  Imp  FreeSelector         (KERNEL.176)
 0003:0446       GetCounterElement
 0000:0000  Imp  GetSelectorBase      (KERNEL.186)
 0003:01F8       GetTickCount
 0000:0000  Imp  GetVersion           (KERNEL.3)
 0000:0000  Imp  GlobalPageLock       (KERNEL.191)
 0000:0000  Imp  GlobalWire           (KERNEL.111)
 0004:01DE       IntCount
 0001:004D       LibInit
 0000:0000  Imp  LoadString           (USER.176)
 0000:0000  Imp  LocalInit            (KERNEL.4)
 0004:01E8       lpOLDISR
 0000:0000  Imp  MessageBox           (USER.1)
 0004:01DC       nInt8Count
 0000:0000  Imp  OutputDebugStr       (MMSYSTEM.30)
 0004:0008       pAtomTable
 0004:0006       pLocalHeap
 0004:0012       PS2_MCA
 0004:000E       pStackBot
 0004:000C       pStackMin
 0004:000A       pStackTop
 0003:0466       qdiv
 0004:0006       rsrvptrs
 0000:0000  Imp  StackEnter           (MMSYSTEM.32)
 0000:0000  Imp  StackLeave           (MMSYSTEM.33)
 0003:0000       tddBeginMinPeriod
 0003:0031       tddEndMinPeriod
 0003:03BB       tddEvent
 0003:0221       tddGetDevCaps
 0003:0216       tddGetSystemTime
 0003:021D       tddGetTickCount
 0003:0278       tddISR
 0003:0199       tddKillTimerEvent
 0003:0263       tddMsToTicks
 0003:0061       tddSetInterruptPeriod
 0003:005D       tddSetInterruptPeriodFar
 0003:00A4       tddSetTimerEvent
 0003:024D       tddTicksToMs
 0003:05B5       ulNormalize
 0004:0010       wEnabled
 0001:0000       WEP
 0000:0000  Imp  WINFLAGS             (KERNEL.178)
 0004:01CD       wMaxResolution
 0004:01CF       wMinPeriod
 0004:0194       wNextID
 0004:01DA       wNextTime
 0004:01D8       wProgTime
 0000:0001  Abs  __acrtused
 0000:0000  Imp  __WinFlags           (KERNEL.178)

  Address         Publics by Value

 0000:0000  Imp  DriverCallback       (MMSYSTEM.31)
 0000:0000  Imp  WINFLAGS             (KERNEL.178)
 0000:0000  Imp  GlobalPageLock       (KERNEL.191)
 0000:0000  Imp  StackLeave           (MMSYSTEM.33)
 0000:0000  Imp  GetSelectorBase      (KERNEL.186)
 0000:0000  Imp  MessageBox           (USER.1)
 0000:0000  Imp  StackEnter           (MMSYSTEM.32)
 0000:0000  Imp  FreeSelector         (KERNEL.176)
 0000:0000  Imp  __WinFlags           (KERNEL.178)
 0000:0000  Imp  GetVersion           (KERNEL.3)
 0000:0000  Imp  AllocCStoDSAlias     (KERNEL.170)
 0000:0000  Imp  LocalInit            (KERNEL.4)
 0000:0000  Imp  LoadString           (USER.176)
 0000:0000  Imp  OutputDebugStr       (MMSYSTEM.30)
 0000:0000  Imp  GlobalWire           (KERNEL.111)
 0000:0001  Abs  __acrtused
 0001:0000       WEP
 0001:0000       Disable
 0001:002A       Enable
 0001:004D       LibInit
 0001:013B       Enable286
 0001:0145       Disable286
 0002:0038       DriverProc
 0003:0000       tddBeginMinPeriod
 0003:0031       tddEndMinPeriod
 0003:005D       tddSetInterruptPeriodFar
 0003:0061       tddSetInterruptPeriod
 0003:00A4       tddSetTimerEvent
 0003:0199       tddKillTimerEvent
 0003:01F8       GetTickCount
 0003:0216       tddGetSystemTime
 0003:021D       tddGetTickCount
 0003:0221       tddGetDevCaps
 0003:024D       tddTicksToMs
 0003:0263       tddMsToTicks
 0003:0278       tddISR
 0003:03BB       tddEvent
 0003:0446       GetCounterElement
 0003:0466       qdiv
 0003:05B5       ulNormalize
 0004:0006       pLocalHeap
 0004:0006       rsrvptrs
 0004:0008       pAtomTable
 0004:000A       pStackTop
 0004:000C       pStackMin
 0004:000E       pStackBot
 0004:0010       wEnabled
 0004:0012       PS2_MCA
 0004:0014       Events
 0004:0194       wNextID
 0004:01CD       wMaxResolution
 0004:01CF       wMinPeriod
 0004:01D2       CurTime
 0004:01D8       wProgTime
 0004:01DA       wNextTime
 0004:01DC       nInt8Count
 0004:01DE       IntCount
 0004:01E4       dTickUpdate
 0004:01E8       lpOLDISR

Program entry point at 0001:004d
